:10019C0008101010101010101010080800000000AB
:0E01AC0000000000082101000000000000001B
:10025B00E51D7020751D011201228F1EE51C651E08
:10026B00FF551EF51BE51EF45FF520851E1CE51BD7
:05027B006002F51A22EB
:10028000E5194518701BF518751901E51A75F00A7E
:100290008475F00A8485F010E51A75F00A8485F0FB
:0202A000112229
:0100030022DA
:1002BF00538E7F5389F0758A18758CFCC28DD28C42
:0502CF00D2A9D2AF220C
:03000B0002009A56
:10009A00C0E0C0F0C083C082C0D075D000C000C02C
:1000AA0001C002C003C004C005C006C007051DE5A3
:1000BA001DB40A03751D000519E51970020518FF1C
:1000CA00AE18BE0109BFF406751800751900051FA0
:1000DA00E51FB40803751F007410251FF8E6FD7CA0
:1000EA00007408251FF8E6FB7A00AF1F1201DE74C0
:1000FA0021251FF8E6FD7C00AF1F120220D007D091
:10010A0006D005D004D003D002D001D000D0D0D080
:08011A0082D083D0F0D0E03266
:1002D4001202A21202BF12025B12028012000380F9
:0102E400F524
:1002A200E5A0541F4480F5A07580FF53A01FE5A070
:0D02B200541F44A0F5A0E4F58053A01F22C6
:0601BA000142000143FFB9
:10022000ED4C600FA8077401088002C333D8FC426C
:1002300042800EA8077401088002C333D8FCF45230
:1002400042E54265436013E5A0541F4480F5A0E5F4
:0A02500042F4F58053A01F854243DD
:01025A002281
:1001C0001129C0F9A4B0999282F880908883C6A1C1
:0D01D000868EFF083A0102040810204080CE
:1001DE00E5A0541F44E0F5A07580FF53A01FE5A0D5
:1001EE00541F44C0F5A0743A2FF8E6F58053A01FB3
:1001FE00EB4A600B74292DF8E6547FF58080077466
:10020E00292DF8E6F580E5A0541F44E0F5A053A093
:02021E001F229D
:10012200E4FFC2A9C2C4D2C2D2B5D2B420B3027F04
:100132000420B2027F0520B1027F0620B0027F07B1
:10014200D2C4C2C2D2B5D2B420B3027F0820B20256
:100152007F0920B1027F0A20B0027F0BD2C4D2C233
:10016200C2B5D2B420B3027F0C20B2027F0D20B1FF
:10017200027F0E20B0027F0FD2C4D2C2D2B5C2B467
:1001820020B3027F1020B2027F1120B1027F122021
:09019200B0027F13D2A975B0FF81
:01019B002241
:0300000002000EED
:0C000E00787FE4F6D8FD758143020055B0
:10001A000202D4E493A3F8E493A34003F68001F226
:10002A0008DFF48029E493A3F85407240CC8C333E7
:10003A00C4540F4420C8834004F456800146F6DFB6
:10004A00E4800B010204081020408090019CE47EA9
:10005A00019360BCA3FF543F30E509541FFEE493AB
:10006A00A360010ECF54C025E060A840B8E493A372
:10007A00FAE493A3F8E493A3C8C582C8CAC583CA9D
:10008A00F0A3C8C582C8CAC583CADFE9DEE780BE55
:0101DD000021
:00000001FF
